:10000000612864001720031801282220A801083065
:10001000A300232017200318A80AAB1EA801A20CD6
:10002000A30B0928AB1AA2132320220808003A08C0
:100030008400380884178004841300052B1B3806BD
:10004000FF3E080037172B081F39003EA1002A0881
:10005000083E0318A10A371F40283713A0000230BA
:1000600057204028A301A200FF30A207031CA307CA
:10007000031C5C280330A100E53040203428A10196
:10008000F63EA000A109031C4B28FE300000A0078B
:1000900003184628A0076400A10F45280000201877
:1000A00051282018532808000310A10CA00CFF3E73
:1000B0000318542820085C28831303138312640058
:1000C000080007309F006400851CB1286400851C6F
:1000D0006A2866280330A300E83033206400851CBA
:1000E0007328BD017F29051583160511053083127C
:1000F000BA000130B8002030AA004030AB00012027
:100100003A3C031D7F2801202A3C031D7F28012043
:100110003D3C031D7F2801204A3C031D7F28012010
:100120003D3C031D7F280120313C031D7F28012019
:10013000653C031D7F280120BC00831601309B0015
:1001400083123C0883169A0004309C0055309D00B1
:10015000AA309D009C149C01831205118316051181
:100160008312831601309B0001309C000130831202
:10017000322083161A088312BC0085158316851158
:1001800083120530BA000130B8002030AA00403098
:10019000AB000120413C031DC9280120643C031D24
:1001A000C92801202B3C031DC92801202B3C031D1D
:1001B000C9280120543C031DC92801207E3C031D91
:1001C000C9280120213C031DC9280120C100BE010E
:1001D00064003E084102031C7E290530BA0001304C
:1001E000B8002030AA004030AB000120C0006400FD
:1001F0003E083C02031D7C29640080304002031C41
:1002000008298030C00286178316861383120C29B2
:100210008613831686138312640040304002031C49
:1002200018294030C00206178316061383121C29B2
:100230000613831606138312640020304002031C49
:1002400028292030C00286168316861283122C2994
:100250008612831686128312640010304002031C3B
:1002600038291030C00206168316061283123C2964
:100270000612831606128312640008304002031C23
:1002800048290830C00286158316861183124C292E
:100290008611831686118312640004304002031C09
:1002A00058290430C00206158316061183125C29F2
:1002B0000611831606118312640002304002031CEB
:1002C00068290230C00286148316861083126C29B6
:1002D0008610831686108312640001304002031CCE
:1002E0007729C00306148316061083127B29061093
:1002F000831606108312C128BE0FE828C1286400A7
:10030000851C83297F2964003D080C3C031D892935
:10031000BD0164003D08003C031DAE290610831694
:100320000610831286108316861083120611831618
:100330000611831286118316861183120612831604
:1003400006128312861283168612831206138316F0
:1003500006138312861383168613831264003D08E6
:10036000013C031DB729061483160610831264008E
:100370003D08023C031DC429061083160610831293
:10038000861483168610831264003D08033C031D07
:10039000D12986108316861083120615831606113E
:1003A000831264003D08043C031DDE2906118316F8
:1003B00006118312861583168611831264003D0888
:1003C000053C031DEB298611831686118312061640
:1003D00083160612831264003D08063C031DF829AB
:1003E000061283160612831286168316861283124D
:1003F00064003D08073C031D052A861283168612F9
:100400008312061783160613831264003D08083C06
:10041000031D122A061383160613831286178316EA
:100420008613831264003D08093C031D372A061415
:1004300083160610831286148316861083120615FF
:1004400083160611831286158316861183120616EB
:1004500083160612831286168316861283120617D7
:1004600083160613831286178316861383120515C7
:100470008316051183128515831685116400831276
:100480003D080A3C031D642A0610831606108312D9
:1004900086108316861083120611831606118312A6
:1004A0008611831686118312061283160612831292
:1004B000861283168612831206138316061383127E
:1004C000861383168613831264003D080B3C031DBC
:1004D000892A061483160610831286108316861046
:1004E0008312061583160611831286118316861150
:1004F000831206168316061283128612831686123C
:100500008312061783160613831286138316861327
:1005100083120130BF0064001A303F020318992A89
:10052000143032206400851C972ABD0A7F29BF0F32
:100530008B2A0511831605118312851183168511E7
:10054000640083123D080A3C031DC62A0614831664
:1005500006108312861483168610831206158316DE
:1005600006118312861583168611831206168316CA
:1005700006128312861683168612831206178316B6
:1005800006138312861783168613831264003D08B0
:100590000B3C031DEB2A06108316061083128614EB
:1005A0008316861083120611831606118312861590
:1005B000831686118312061283160612831286167C
:1005C0008316861283120613831606138312861768
:1005D0008316861383120130BF0064001A303F0275
:1005E0000318FB2A143032206400851CF92ABD0A46
:0C05F0007F29BF0FED2A7F296300FC2A41
:02400E00463F2B
:024202000000BA
:00000001FF
